S1048000007B
S123C000C787C769C790C7C4C76FC777C77FC7D2C7EAC7E2C7F2C844C83AC82EC833C84D42
S123C020C865C8B3C875C885C895C93BC95BC967C97BC78DCA5EC991C9A6C99BCABACAC614
S123C040CAD1C9C3C9AFC9CDC9D7C9E7CA28CA54CA63CA7FCA8ECA9DCA34CA44CA19C9FF5B
S123C060CAE6CAEACAF0CB01CB14CB07CB4ACB1CCB5ACBBDCBD2CBE0CBF2CB95CB9FCB7866
S123C080CBA8D77AD726D750D768D78DD7A0D7B2D7BDD7D5D7FAD80AD7ABD825D839D84472
S123C0A0D81AD84FD85AD865D877D885D893D735D8BBD8E0D8CBD8A1DCF2DDD0DDD4DE1947
S111C0C0DA8ECBABCBB4DA67DA9DDAAE0000D1
S123C500FCFF0227358E00FFBDE0ED1AB3FF022608CC0000FDFF022021BDDB82CEC52DBD09
S123C520DCE1B67F0084C088C027F720134D454D4F5259204641554C54008EFEFF7F003C6D
S123C5408D392016B67F0084038103260D8E00FF0FBDE0EDFDFF027EE089B67F008480889C
S123C5608027037EC712B680004A26F7CC8001CEC300ED008600A7097EC712CE002A4FA7D3
S123C58000088C003926F8CE1000860AB77F00970E86FF9722972397249725CC07C0DD265E
S123C5A01C39801D282086B0A72B860CA72D86079739BDDB82CC0000DD0CDD12DD14860835
S123C5C0970BCCC110DD16DD18DD1A8620B7C6F8CEC300C6208640A7098FC300108F5A26C0
S123C5E0F6CEC300DF08CCC200ED00CCFE00ED04C30001ED02830100ED06860AA708862084
S123C600A709EF0CEF0EDC0CC30001DD0CED0ABDDAAECEC639A6002706BDDB540820F6CE25
S123C62010001C200118CE3000180926FC1D20011D0008CC0000DD2639496E74657261631F
S123C6407469766520432020205620322E383120392F32382F39330A008D6B8D7481612585
S123C660F881732604863E2068368D513C18388D4C328172270D8177270F81632711816255
S123C680271B39A6008D4A2010188FE700200A188FA400A700EA00E700863E2034188F37FD
S123C6A03C32331B331B97015D270C8D19A7009B019701085A26F496018D1620DC8D073647
S123C6C08D0416328F39B6102E842027F9B6102F39F6102EC48027F9B7102F39DE08A60874
S123C6E0970A1AEE00EE0218E600F7C6F11808FCC000FDC6F6BDFFFF20ED8620B7C6F8DC9D
S123C700088FED021AEF00A60981402604EE0CDF0839963C260CCE10001F2E2005BDC659A2
S123C72020F0120B02ECDE08EE0EDF088CC3002607DC1EC30001DD1EA609810026D4BDC62F
S123C740DC810027CD814027C9812027048602200286048D0220BB9701940B910126013940
S123C76096019A0B970B7EC6D1EC02A300201CEC02A400E4012014EC02AA00EA01200CECAF
S123C78002A800E8012004EC00E302ED020808398D26A601E6033DDD00A600E6033DDB00D1
S123C7A0D700EC013DDB00D7007D000727064F5F930020D7DC0020D37F00078D6308088DF7
S123C7C05F090939BDC7B8EC023CEE0002DF003820D7EC00A3022705CC000020AECC000123
S123C7E020A9EC02A3002EF520EEEC02A3002DED20E63CEC002B1C260438080839373686EC
S123C80005B7C807EC02380027030926FA380808ED00394F5FA30037368604B7C80720E4D0
S123C8206D002A094F5FA300ED007300073963006301394F5FA300ED0039EC002705CC0008
S123C84001ED0039EC0027F64F5FED0039EC02E306DD00E601E905A600A904ED04DC00ED3A
S123C86006C6043A39EC06A302DD00E605E201A604A20020E6EC06A302E605E201A604A22C
S123C880002D1E2025EC02A306E601E205A600A2042D0E2015EC06A302260FEC04A300265E
S123C8A009C6063ACC0001ED0039C6063ACC0000ED00397F0007BDC9513CC6043ABDC95106
S123C8C0CE0000DF0038A603E6073DDD02A603E6063DD301DD01960089009700A602E607EE
S123C8E03DD301DD01960089009700A603E6053DD300DD00A602E6063DD300DD00A601E600
S123C900073DD300DD00EC033DDB00D700A602E6053DDB00D700A601E6063DDB00D700A697
S123C92000E6073DDB00D700C6043ADC02ED02DC00ED007D000727028D0139CC0000A30298
S123C940DD00C600E2018600A200ED00DC00ED02396D002A058DE47300073918EC00180850
S123C96018080909ED003918EC020909ED0018EC00180818081808180820E718E600183A7B
S123C98018A60009A70018095A26F518E600183A393CCDEE00E600384F20C38FCDEE00EE87
S123C9A0028F0909ED008FCDEE00EE008F20AF18E6003C3AEC00DD00EC02380909ED00DC0F
S123C9C000209D18E6003C3AEC003820933CA601CDEE00A70020083CEC00CDEE00ED0018F6
S123C9E0083818080808393CEC00DD00EC02CDEE00ED02DC00ED0038C6043A57183A39EC1A
S123CA0000DD00EC02D70718E6003C3AD607ED02DC00ED0038080820C9EC00D70118E6006D
S123CA203C3AD601ED0020B9A6013CEE02273FA70038202AA601B7CA403CEE0227301C0076
S123CA40FF38201AA601B7CA503CEE0227201D00FF38200AEC003CEE022713ED0038080871
S123CA60080839EC00DD00EC023CEE0426063886057EDE25ED02DC00ED0038080820DFEC29
S123CA80003CEE0227E8E70038ED02080839EC003CEE0227D9ED0038ED02080839EC00DDC2
S123CAA000EC023CEE0427C6ED02DC00ED0038EC02ED04DC00ED020808393CEE0027AFE6A0
S123CAC0004F38ED00393CEE0027A3EC0038ED00393CEE002798EC00DD00EC02380909ED90
S123CAE002DC00ED003918EE00391AEE00080839EC00260618EE00080839180818080808E7
S123CB0039EC0026EF20F3EC0027EFCC0001ED0018EE0039EC0026E218EE0039EC00DD00CD
S123CB2018EC00DF04D3048F1AEE002705DC00ED0039DE088640A7098621B7C6F8EC0C1AE4
S123CB40EE0E8FCDEF0C1AEF0E3918EC00DF00D3008F1AEE0027DB080839EC00DD00EC02DF
S123CB60DD0218EC00DF04D3048F1AEE0227C3DC00ED00DC02ED0239DF00DE08DC00A30678
S123CB80CDA300250718081808DE00391809DE0086047EDE258F18E3008F18081808393CC6
S123CBA0323318E3007EC95EEE0039EC00DD3A0808180839DC3A0909ED00180839EC003C43
S123CBC0EE021AA300382427E302C30002ED02080839EC003CEE021AA3003824120520E8EF
S123CBE0EC003CEE021AA300382404050520D97EDE1FEC003CEE021AA3003824F218A6009D
S123CC0018083D20C33CBDD696CE00003CDF3DDF3F7F00411830CDEE06A600BDCD5D252884
S123CC20812D260B73004108A600BDCD5D2519812E260B08A600BDCD5D24037ECCCB313177
S123CC40BDD6A038860F0D39A600BDCD5D2477BDCCDC0824F37C003DA60008BDCD5D25F576
S123CC60812E260AA600BDCD5D24030820F681452707816527037ECD1F08A600BDCD5D25D7
S123CC8015812D2706812B270520B318630008A600BDCD5D24A8803018A70108A600BDCD71
S123CCA05D241418E601585818EB015880301B18A701088126228718A601186D002A01403E
S123CCC09B3D973D2059812E26A408A600BDCD5D249C8D0808258D7A003D20EF963E97439A
S123CCE0DC3FDD440579003E252C0579003E2526D34436963E9943973E32251A0579003EE1
S123CD00DD3F2512E600C0304FD33FDD3F963E89002503973E39DC44DD3F9643973E39CDE6
S123CD20EF06CE003DBDCD88272C963D18A7018696973DBDCD69186D01271B2A0BCECD93E9
S123CD40BDD6C91860012006CECD97BDD6C9BDCDA7186A0126F83131BDD6A0383981302598
S123CD6006813922020D390C39CE003D8D1A27147D003E2B0FDC3F7A003D270A0579003E9F
S123CD802AF5DD3F0C390D393736EC002602EC023233393DCCCCCD41200000BDD043BDD656
S123CDA096BDCF12BDD6A07D003D27057D0042260ACC00009741DD3DDD3F399641984697D4
S123CDC041963D9B422A0924168606CEFFFF2009250D8607CE0000DF40DF3DDF3F0D398BB9
S123CDE082973DCE00003C3C30BDCE206D002B0B69036902690169007A003D6D032A13A661
S123CE00024CA702260CC601E3002404467C003DED0038DF3E329740317D003D27B45F396B
S123CE209645D6403DA7019644D6403DE300ED009645D63F3DE300A70324026C026F006FEF
S123CE40019643D6403DE302ED029644D63F3DE302ED0224026C019645D63E3DE302ED023A
S123CE6024026C019643D63F3DE301ED0124026C009644D63E3DE301ED0124026C00964324
S123CE80D63E3DE300ED0039BDD696CED3C2BDD6C97D00412703730046BDCF44BDD6A04F59
S123CEA0D63DC17F24035F201B53C3FF902F178FDC3E2001040926FC7D00412A074353C32E
S123CEC000012A020C3986090D39CC0000DD004FD63DC17F24035F203353C3FFA02F2F8F41
S123CEE096405FDD00DC3E2007047600007600010926F67D00412A1473000073000143534C
S123CF00DE0008DF002605C300012A020C3986090D39BDD32ACE0045964280972A1BC60349
S123CF208B082A096F00095A26F66F0039C6804A2B035720FAE400E7008D028D0796468810
S123CF40FF974639963D260EDC42DD3DDC44DD3F964697415F397D004227F9D641D846904D
S123CF60422510811822ED183C36CE004318CE003E201740811822D0183C369642973D9601
S123CF80469741CE003E18CE004317363636A8003617A8013617A8023630A606E706168453
S123CFA0074CC4185454543AE6034A27095666026601660020F45618A602A900974018A6B2
S123CFC001A901973F18A600A902973E30A6062B15245A76003E76003F7600407C003D26F6
S123CFE04CCCCDC92053251B73004170004024087C003F26037C003E70003F24037C003E0E
S123D00070003E7D003E2B252613963D80082326973DDC3F27207F0040DD3E20E67A003DA9
S123D020271478004079003F79003E2AF01AEE07C6093A355F39CCCDD21AEE07ED07C60750
S123D0403A35399646984197417D0042260586087ECDCB7D003D26055F7F004139963D9069
S123D0604224052B057ECDD22B1F8B7E973DDC3E93432B182606964090452B10DC3E0476F4
S123D0800040DD3E7C003D26037ECDC9DC3EDE430826010903183C18DE3EDF3E3CCE000016
S123D0A03C3C309645D63F3DA703BDCE4A18DF3EDC3FA301DE4303DF3F7F003E3838323350
S123D0C01838D33EDD3E5F393CCE003DBDCD88260738CC3000ED0039DE3D3CDE3F3C9641D1
S123D0E036BDD696CE00003C3C3C1830CDEE0F86207D004127057F0041862DA70008CDEFCB
S123D10000CED232BDD6C9BDD2362E19CED22EBDD6C9BDD2362E16186A02CECD97BDD6C98C
S123D120BDCDA720DC186C02CECD9320F0CED3C2BDD6C9BDCF44D63DC07F50CB17200A7449
S123D140003E76003F7600405A26F4860118A70318A6028B082B0A810824064A18A7038698
S123D16002800218A702186D032E15862ECDEE00A70008186D0327058630A70008CDEF00A8
S123D180CED219860718A705186F04DC3FA301DD3F963EA200973E2505186C0420EDDC3FF6
S123D1A0E301DD3F963EA900973E18A6048B303CCDEE00A70008186A032605862EA70008E3
S123D1C0CDEF0038080808186A0526BCCDEE0009A600813027F90818E602272A8645A700D0
S123D1E008862BA7005D2A0550862DA70008CDEF004FCE000A02378FCB30CDEE00E700083D
S123D20033CB30E700086F00383838BDD6A032974138DF3F38DF3D38390F42400186A000C6
S123D22027100003E800006400000A000001497423FE4B18967F96462A12D6412A0EDC427E
S123D2401A933D2617DC441A933F20109141260CDC3D1A93422605DC3F1A93440784F42481
S123D260028A080639CE008EC3000026057ECDD209052AFCDD3E7F00408F9741D73D5F394F
S123D2804D2AE24353C30001CEFF8E20DBCE009EC30000261118DE0026037ECDD20978005E
S123D2A00179000059492AF5DD3E960097408F9741D73D5F394D2AD57300007300014353CB
S123D2C0DE0008DF002603C30001CEFF9E20C1CE003DBDCD882601397D00412A04860A0D46
S123D2E039BDD696860436DE3F3CDE3D3C18308D399642807E4C2A03442003448B7E97426E
S123D300BDD043BDCF447A003D8D1F18EC00DD3D18EC02DD3F186A0426E6DC42DD3DDC44DC
S123D320DD3F383831BDD6A05F39DC3DDD42DC3FDD449641974639BDD696CED491BDD6C948
S123D340BDD043BDD6A0DC3D1A8385B32B0B7D004126037ECDC97ECDD2BDD6969641367FD5
S123D3600041BDCF12DC4227068086544C26FC5C37CED3A6BDD656CED3A2BDD6C92003BD75
S123D380CDA7306A0026F832324D2A0CBDD32ACED5EABDD6B0BDD043BDD6A05F39BDD69628
S123D3A020EA402DF8543638EF1D37D00D0139500D013AB60B613C0888893D2AAAAB3E2AAB
S123D3C0AAAB3F0000003F8000003F800000FFBDD3EBBDCDA77ED3468D11BDD696CED491FB
S123D3E0BDD6C9BDCDA7BDD6A05F3996412704860C0D39963D27F8BDD6963C3C30BDD6E1C0
S123D4004FD63DC07F2A0143BDD280CED48DBDD6C9BDCDA730BDD6C9BDD6E1867F97423C14
S123D4203C30BDD6EFCED5EABDD6B0BDCF4430BDD6C9BDD6E1CED489BDD6B0BDCF4430BD2F
S123D440D6C9BDD04330BDD6E1BDD32ABDCDA7CED46CBDD65630BDD6C9BDCDA7383830BDB9
S123D460D6C9BDCF443838BDD6A05F393E1D89D93E3A2E8C3E638E393E9249253ECCCCCDC6
S123D4803F2AAAAB40000000FFBF8000003F3172183EDE5BD9860E0D39860D0D39BDD69626
S123D4A09641367F0041CED5EABDD6C9BDD2362F07BDD39D86FF20014F363C3C30BDD6E143
S123D4C0BDD32ABDCDA7CED4F4BDD65630BDD6C9BDCDA73838324D270CCED4F0BDD6C9739E
S123D4E00041BDCF44BDD640329741BDD6A05F393FC90FDBBCE2DD1B3D70F0F1BD88888903
S123D5003D9D89D9BDBA2E8C3DE38E39BE1249253E4CCCCDBEAAAAAB3F800000FFBDD696AE
S123D5204F2005BDD69686F036CED608BDD6C92003BDCF44964126F92003BDCF39BDD23600
S123D5402EF88D61240930A6002B04880FA7008D54240930A6002A04880FA7008D472407F4
S123D56030A60088F0A700CED64EBDD6C9BDCDA7BDD32ABDCDA73C3C30BDD6EFA6042A0545
S123D580CED5EF2003CED5DABDD65630A6044724037300414D2B06BDD6C9BDCDA7383831C4
S123D5A0BDD6A05F397A0042BDD2362E020C397C0042730041BDCF447A00420D39BDCF12C4
S123D5C0DC3DDE42DD42DF3DDC3FDE44DD44DF3F9641D6469746D7415F393638EF1DB95054
S123D5E00D013C088889BE2AAAAB3F800000FF37D00D01BAB60B613D2AAAABBF0000003F1E
S123D600800000FF40490FDB43B40000BDD696BDD32ABDD523BDD5C0BDD51DBDD043240789
S123D620BDD6A0860B0D39BDD6A05F397FFFFFFFBDD696CED64EBDD6C9BDCDA7BDD6A03981
S123D640BDD696CED65220EECED6047ED6B03C8EFA3142652EE18FDE3D3CDE3F3C8F96419D
S123D660363CCC0000DD3DDD3FDD40201030A6029746EC03DD44EC05DD42BDCDA730EE00C1
S123D680BDD6C9BDCF4438C6043A3CA6004326DD30C6073A3539383C3C8F3037367ED6EF32
S123D6A0300808BDD6C938313131316E00CED5EA7F0041EC02DD3FEC0005240373004197A6
S123D6C03D27020D56D73E5F397F0046EC02DD44EC00052403730046974227020D56D743AC
S123D6E039DC3FED02DC3D58D1414656ED0039DC44ED02DC4258D1464656ED00397F004180
S123D7005F397D003E2705CC7F80DD3D4F5FDD3F397D003E27037300415F39BDD6C9080801
S123D7200808BDD6B0393C183CEC00BDD280183838090920AC3C183C0808BDD6B00909EE85
S123D74000BDD0C8183838EC00ED0408080808393C183CBDD6B0BDCECA18383824037EDE7F
S123D76025ED00DC00ED02393C183CEC02DD00EC00BDD2B51838387ED6E13C183CBDD6B074
S123D780BDCE9F18383824037EDE25205D3C183CBDD71BBDCF44183838080808087ED6E1C2
S123D7A03C183CBDD71BBDCF3920EBA6008880A700393C183CBDD71BBDCDA720093C183C9F
S123D7C0BDD71BBDD04318383824037EDE25080808087ED6E13C183CBDD71BBDD2361838ED
S123D7E038260CCC0001080808080808ED00390808080808086F006F01393C183CBDD71B11
S123D800BDD2361838382BDB20E53C183CBDD71BBDD2361838382ECB20D53C183CBDD71BF3
S123D820BDD3CF20A13C183CBDD6B0BDD2CF18383824037EDE257ED6E13C183CBDD6B0BD9E
S123D840D34620EA3C183CBDD6B0BDD33720DF3C183CBDD6B0BDD3EB20D43C183CBDD6B0F3
S123D860BDD3D820C93C183CBDD6B0BDD49D0736BDD630320620B73C183CBDD6B0BDD6409D
S123D880BDD51D20A93C183CBDD6B0BDD640BDD523209B3C183CBDD6B0BDD640BDD60C2091
S123D8A08D8602E6019D47080839BDDB9AA600BDDC7EA601BDDC7E08082003BDDB9AA60083
S123D8C0BDDC7EA601BDDC7E080839BDDB9A3CEE008602E60027059D470820F738080839AC
S123D8E0183CDF00BDDAFA1A830051240C8621B7C6F8DE001838180939DE00DC00C300021F
S123D900E300DD02830002DD04DE02EE000808A60026037EDA55812527037EDA4308A60068
S123D9208166261BDF02DE0409093CBDD6B0380909DF04CEC100BDD0C8CEC1007EDA3581B9
S123D94064267DDF0218CEC100DE040909DF04EC022A0C862D18A7001808CC0000A302CE68
S123D960000A02378FCE000A02378FCE000A02378FCE000A02378FCE000A0237183C3886CE
S123D98001335D27064FCB30E70008334D27045D27064FCB30E70008334D27045D27064F9A
S123D9A0CB30E70008334D27045D27064FCB30E7000833CB30E700085FE700CEC100207584
S123D9C08178262ADF02DE040909DF04A602BDDC64BDDB42257217BDDB42256CA603BDDC68
S123D9E064BDDB42256217BDDB42255C206181632611DF02DE040909DF04A603BDDB4225F0
S123DA0047204C8162261EDF02DE040909DF04E60318CE00085886308900BDDB42252918C2
S123DA200926F2202A8173261ADF02DE040909DF04EE020808A6002708BDDB42250A082085
S123DA40F4200CBDDB422409860ABDDB542006DE02087ED90FDE00DC00C30002E3008FCCEE
S123DA600000ED001838393CDC14C300011A931426FBC30001CE0000081A931426FA8F3818
S123DA800909ED00CC000C0909ED007EC790090909090FDC14ED02DC120EED0039EC0008AF
S123DAA0083C183CEE00AD00183838ED00390F3C183CB6103C84402605CEFF002003CEBF74
S123DAC0003CC6C03A18CEE0FF1AEF0008083C32324D26F538CCC500EDFECCDE9FEDE2CCC8
S123DAE0DE92EDE0CE10006F226F248630A7211C23181C22181838380E39960B840827078E
S123DB00CC00F0DD062016DC1893162307830001DD062009CC00F09316D318DD06960B847D
S123DB20102705CC00F02012DC1A931623058300012007CC00F09316D31A1A93062302DC3F
S123DB4006393736BDDAFA1A83000224040D323339322001370F3CDE16088CC2002603CEFC
S123DB60C110DF16A700960B840827119C18260DDE18088CC2002603CEC110DF1838330C66
S123DB800E398D79CC00389D47C60C9D478D198601970F8608971C4F971DCC00019D47C608
S123DBA0069D47C68F9D4739CC00409D478602CEDBBDE6009D47088CDBFD26F639000A1F73
S123DBC01F0E04000000001111110F010E00000000000C040800000F11110F010E00000C4C
S123DBE00C000C0C0000000C0C000C0408020006020202120C00000A0E04000000CEDC12C9
S123DC0018CE0047A60018A7000818088CDC6426F339FF0096CE10000F1D3C201D0010B749
S123DC2000986F078104260F8601B710041C0010A6031D001020228601B710041C0010A65E
S123DC40031D0010848026EF86FFA707B60098A704E7031C00101D00101C3C20FE00960EEE
S123DC603900000036840F8B30813A2B028B071632444444448B30813A2B028B0739BDDC0A
S123DC8064371686029D47339D4739CE000A02378FCE000A02378FCE000A02378FCE000A5B
S123DCA002378FCE000A02379D47CC00019D47CC00079D47CC008F9D47860233CB309D4762
S123DCC033CB309D47C62E9D4733CB309D4733CB309D4733CB309D47C66D9D47C6739D47EC
S123DCE039CC00029D478602E60027059D470820F739183CDF00CC7FFFDD04CEC3001AEE68
S123DD000E188CC3002607CCE400DD06200518EC04DD06EC0693063CDE00A300382B091AEC
S123DD2093042E04DF02DD04188CC3002705183C3820CBDC041A837FFF260486012015CE9B
S123DD40C310A609814027158FC300108F8C620026F08602DE00183818097EDE253C183867
S123DD60DE02EE0E1AEF0CCDEF0EDE021AEF0ECDEF0CEC0683000118ED04C30001DE00A361
S123DD800018ED06A60318A708EC0418ED00860018A709DC0CC30001DD0C18ED0ADC00E35E
S123DDA006C30008EE068F09DF0018DF0218EE0436A60018A7003209180983000126F1DEB0
S123DDC00218081AEF02DE0009DC0CED00183839862020513CEC00DD00CEC300EC0A1A937D
S123DDE000270EEE0E8CC30026F238CC0001ED00399C082604387ECB32183C8640A709868B
S123DE0021B7C6F8EC0C1AEE0E8FCDEF0C1AEF0E183838CC0000ED00398621B7C6F8391805
S123DE2009860320003CDE084D2602861FA70997018621B7C6F8960181202431CEDE6FA63E
S123DE40002708BDDB4225F70820F44FD601C00A25034C20F9CB0A8B30BDDB4225FB178BD4
S123DE6030BDDB4225FB860ABDDB4225FB38390A52554E54494D45204552522000CE100044
S123DE80DC28E316ED161D237FB610008880B710003BCE1000DC26E31EED1E1D23F73BCEC3
S123DEA01000CC07D0E31CED1C1D23EFA622368408A7220EDE1408DF142605DE1208DF1212
S123DEC07A000A26058621B7C6F886049D47848027037EDFAC9615843F2640960F810122B1
S123DEE03A0F4FC6CF9D47DC1E1A8300642D0BCC0000DD1E961C880C971C961C84082704B1
S123DF00C6002002C60786029D474FD611C1102502CB30CA809D470E7EDFAC9639840126F4
S123DF20037EDFAC960F8102245EDE1A9C16277C088CC2002603CEC110DF1AE600960F81B7
S123DF40002634C10A26068601970F205F9611811F27594C9711811126074F37C6C09D4756
S123DF6033C120250CC17F2208CEE00CC0203AE60086029D4720358101260DD710FCDFFA02
S123DF809D478602970F2024810A2712CEDFFAD60F3AEC009D47960F8B02970F200E860041
S123DFA0970F86019711D610C10A26B5D60E96398404273E96224824068B01C8102002CAE2
S123DFC010972296234824068B01C8202002CA20972396244824068B01C8402002CA40978C
S123DFE02496254824068B01C8802002CA809725C8F0F77F0032B710223B0001000600CF76
S123E000020000020011495557777FFF202122232425262728292A2B022D2E2F30313233E9
S123E02034353637383904053C3D3E3F404142434445464748494A4B4C4D4E4F50515253D8
S123E0405455565758595A5B5C5D5E5F60616263646566036869066B6C6D6E6FF0F1727314
S123E0607475767778017A7B7C7D7E7F18CE03E8180926FCCE10001F000433CC1BE61F002E
S123E080042C83000126F7203937368D56CC00029D47CEE0B78602E60027059D470820F74E
S123E0A032BDDC7E32BDDC7E8602C6299D47CE10001C28204F06CF2A48616C7465642A2043
S123E0C028008D1FCEE0D3BDDCE1CE10001D23FB8D163B2D504F57455220474C49544348E1
S123E0E02D20008601979439860E979439CE80004F5FE3008FC300028F8CFF0226F4393B0F
S123BFC0E0FFE0FFE0FFE0FFE0FFE0FFE0FFE0FFE0FFE0FFE0FFE0FFE0FFE0FFE0FFE0FF6D
S123BFE0DE92DE9FE0FFE0FFE0FFE0FFE0FFE06CE0FFE0FFE0FFE0FFE0FFE0FFE0FFC500CB
S123FFC0E0FFE0FFE0FFE0FFE0FFE0FFE0FFE0FFE0FFE0FFE0FFE0FFE0FFE0FFE0FFE0FF2D
S123FFE0DE92DE9FE0FFE0FFE0FFE0FFE0FFE06CE0FFE0FFE0FFE0FFE0FFE0FFE0FFC5008B
S105FF020000F9
S105FF000251A8
S9030000FC
